:100000000C94F4050C943C060C943C060C943C06B1
:100010000C943C060C943C060C943C060C943C0658
:100020000C943C060C943C060C944F240C942A210E
:100030000C9401210C943C060C943C060C943C0658
:100040000C943C060C943C060C943C060C943C0628
:100050000C943C060C94DB200C943C060C943C065F
:100060000C943C060C94EF280C943C060C943C0633
:100070000C943C060C943C060C943C060C943C06F8
:100080000C943C060C943C060C943C060C943C06E8
:100090000C943C060C943C060C943C060C943C06D8
:1000A0000C943C060C943C060C943C060631FF096B
:1000B00074A1010975150026FF00952075088102BD
:1000C0000976150026FF00952075089102C00501EC
:1000D0000902A1010901A1008501050919012908E9
:1000E00015002501950875018102050109300931C6
:1000F0001581257F95027508810609381581257FB0
:10010000950175088106050C0A38021581257F9531
:100110000175088106C0C005010980A1018502168C
:1001200001002637001A81002AB700751095018159
:1001300000C0050C0901A1018503160100269C02DF
:100140001A01002A9C02751095018100C005010961
:1001500006A101050719E029E71500250195087595
:10016000018102050819012905950575019102957E
:1001700001750391010507190029F715002501955F
:10018000F875018102C025730D0A002563002B0D4F
:100190000A00760D0A0024242400456E74657269F5
:1001A0006E6720636F6E666967206D6F6465202ED1
:1001B0002E2E0A002D2D2D0D0A0045786974696ECA
:1001C0006720636F6E666967206D6F6465202E2EF1
:1001D0002E0A00522C310D0A0053522C5A0D0A00DF
:1001E000522C310D0A0053592C464646340D0A0054
:1001F00053482C303033430D0A00537E2C360D0A01
:100200000053572C383030300D0A00534D2C340D2C
:100210000A0053532C4B6579626F6172642F4D6FE6
:100220007573650D0A00532D2C546D6B42540D0AE5
:100230000053462C310D0A00555342206D6F646502
:100240000A004175746F206D6F64650A00253032B5
:10025000750A00253032753A00253032753A004271
:1002600041543A2025756D560900757074696D65A5
:100270003A202530327520253032753A25303275D6
:100280003A253032750A00564255533A2025580A0D
:100290000052656D6F746557616B657570456E6171
:1002A000626C65643A2025580A000A003F004C4FF2
:1002B000570044495343484700434841524700468A
:1002C000554C4C00626174746572793A2000555344
:1002D000422053746174653A2025730A00636F6E7F
:1002E0006669675F6D6F64653A2025580A00726E13
:1002F00034325F6175746F636F6E6E656374696EBF
:100300006728293A2025580A00726E34323A20258F
:10031000730A00666F7263655F7573623A202558D1
:100320000A0070726F746F636F6C3A2025730A0055
:100330000A2D2D2D2D2D20524E2D343220696E6622
:100340006F202D2D2D2D2D0A00753A2020202020E4
:100350002020746F67676C6520466F726365205557
:100360005342206D6F64650A00703A2020202020DF
:10037000202070616972696E670A00536C636B3A82
:1003800020202020524E2D343220696E697469611C
:100390006C697A650A0044656C3A2020202020654B
:1003A0006E7465722F6578697420524E2D34322038
:1003B000636F6E666967206D6F64650A00623A203C
:1003C0002020202020206261747465727920766F6D
:1003D0006C746167650A00693A2020202020202083
:1003E000524E2D343220696E666F0A000A0A2D2D96
:1003F0002D2D2D20426C7565746F6F746820524EE0
:100400002D34322048656C70202D2D2D2D2D0A00A5
:1004100025583A2530386225730A000A20203031E9
:100420003233343536370A004C45443A20253032D1
:10043000580A00253032753A253032753A25303267
:10044000750925756D560A004C4544207374617416
:1004500075733A20253032580A0020253032580072
:100460002563005B735D004B6579626F6172642088
:1004700073746172740A00524E2D343220696E69B1
:10048000740A000A55534220696E69740A00090211
:100490005400030100A0320904000001030101001F
:1004A0000921110100012239000705810320000103
:1004B00009040100010301020009211101000122C8
:1004C0007F00070582030800010904020001030000
:1004D00000000921110100012222000705830320E9
:1004E00000011201100100000008EDFE424204016B
:1004F000010200011203480048004B0042002000A6
:100500006D006F00640000000E0374002E006D008B
:100510002E006B002E00000004030904737973742D
:10052000656D3A20253034580A00636F6E73756D1F
:1005300065723A20253034580A000A0025750036C5
:100540003A20776865656C5F74696D655F746F5F8D
:100550006D61783A20000A00257500353A207768E9
:1005600065656C5F6D61785F73706565643A2000E6
:100570000A00257500343A2074696D655F746F5FF9
:100580006D61783A20000A00257500333A206D61CC
:10059000785F73706565643A20000A002575003243
:1005A0003A20696E74657276616C286D73293A2001
:1005B000000A00257500313A2064656C6179282AAB
:1005C00031306D73293A20000A092D2056616C756F
:1005D0006573202D0A004D3E004D25643E20003FEE
:1005E000007365742064656661756C740A00433E2F
:1005F00020000A002530325820006B6579626F6157
:1006000072643A20004F6E6573686F743A207469A3
:100610006D656F75740A001F141A16041D1B0620E1
:100620002115080709190522231C170A0B11801E22
:10063000352B39797A7B2C2425180C0E0D108074FB
:100640002A31287C7D7E7F26271213330F36802D9A
:100650002E302F34383780290A002575002F0025C9
:1006600075005D2800256400200025640020002519
:10067000640020002564007C0025303258006D6F36
:100680007573656B6579205B62746E7C7820792068
:100690007620685D287265702F61636C293A205B53
:1006A000006D6F7573653A205B253032587C256488
:1006B0002025642025642025645D0A000A092D2078
:1006C0004D61676963202D0A643A09646562756744
:1006D0000A783A096465627567206D617472697899
:1006E0000A6B3A096465627567206B6579626F61B0
:1006F00072640A6D3A096465627567206D6F75737F
:10070000650A763A0976657273696F6E0A733A09FB
:100710007374617475730A633A09636F6E736F6CF7
:1007200065206D6F64650A302D343A096C61796516
:1007300072302D34284631302D4634290A506175E7
:10074000733A09626F6F746C6F616465720A6E3A16
:10075000094E4B524F0A000A092D20436F6E736FEA
:100760006C65202D0A4553432F713A0971756974E0
:100770000A6D3A096D6F7573656B65790A003F0004
:100780004E4B524F3A206F66660A004E4B524F3A1C
:10079000206F6E0A0074696D65725F726561643303
:1007A0003228293A202530346C580A006B6579626A
:1007B0006F6172645F6E6B726F3A2025580A006B2E
:1007C0006579626F6172645F69646C653A2025586F
:1007D0000A006B6579626F6172645F70726F746F2B
:1007E000636F6C3A2025580A00686F73745F6B65FD
:1007F00079626F6172645F6C65647328293A2025A1
:10080000580A000A092D20537461747573202D0A4B
:10081000004743433A20372E332E30204156522D85
:100820004C4942433A20322E302E30204156525FFE
:10083000415243483A20617672350A004F5054497C
:100840004F4E533A204C554641204D4F5553454B42
:1008500045592045585452414B455920434F4E531A
:100860004F4C4520434F4D4D414E44204E4B524F2F
:10087000204B45594D41505F53454354494F4E20FD
:10088000343039360A004255494C443A20373163F6
:10089000333437202832303A31343A3037204D6102
:1008A000722031392032303234290A005649443A14
:1008B0002030784645454428742E6D2E6B2E292015
:1008C0005049443A203078343234322848484B4238
:1008D000206D6F6429205645523A203078303130EF
:1008E000340A00444553433A20742E6D2E6B2E205B
:1008F0006B6579626F617264206669726D7761728F
:100900006520666F722048484B42206D6F640A0074
:100910000A092D2056657273696F6E202D0A000A30
:100920006D6F7573653A206F66660A000A6D6F75A4
:1009300073653A206F6E0A000A6B6579626F6172A7
:10094000643A206F66660A000A6B6579626F6172AD
:10095000643A206F6E0A000A6D61747269783A20F9
:100960006F66660A000A6D61747269783A206F6E6C
:100970000A000A64656275673A206F6E0A000A64AD
:10098000656275673A206F66660A000A0A626F6FD1
:10099000746C6F616465722E2E2E2000433E200021
:1009A0006D6B5F776865656C5F74696D655F746FAB
:1009B0005F6D6178203D2025640A006D6B5F77686C
:1009C00065656C5F6D61785F7370656564203D205F
:1009D00025640A006D6B5F74696D655F746F5F6D90
:1009E0006178203D2025640A006D6B5F6D61785F42
:1009F0007370656564203D2025640A006D6B5F6936
:100A00006E74657276616C203D2025640A006D6B02
:100A10005F64656C6179203D2025640A006D6B5F21
:100A2000776865656C5F74696D655F746F5F6D6134
:100A300078203D2025640A006D6B5F776865656CE2
:100A40005F6D61785F7370656564203D2025640A81
:100A5000006D6B5F74696D655F746F5F6D617820A9
:100A60003D2025640A006D6B5F6D61785F73706572
:100A70006564203D2025640A006D6B5F696E7465B6
:100A80007276616C203D2025640A006D6B5F6465A1
:100A90006C6179203D2025640A00776865726520C5
:100AA00064656C74613A20637572736F723D25647E
:100AB0002C20776865656C3D25640A536565206860
:100AC0007474703A2F2F656E2E77696B6970656448
:100AD00069612E6F72672F77696B692F4D6F757320
:100AE000655F6B6579730A000A092D204D6F757378
:100AF000656B6579202D0A4553432F713A0971754D
:100B000069740A313A0964656C6179282A31306D5B
:100B100073290A323A09696E74657276616C286DC0
:100B200073290A333A096D61785F73706565640AE9
:100B3000343A0974696D655F746F5F6D61780A3569
:100B40003A09776865656C5F6D61785F737065659C
:100B5000640A363A09776865656C5F74696D655F2C
:100B6000746F5F6D61780A0A703A097072696E7409
:100B70002076616C7565730A643A09736574206444
:100B8000656661756C74730A75703A092B310A6475
:100B90006F776E3A092D310A706775703A092B31FB
:100BA000300A7067646F776E3A092D31300A0A7324
:100BB00070656564203D2064656C7461202A206D39
:100BC00061785F7370656564202A2028726570659E
:100BD0006174202F2074696D655F746F5F6D61783B
:100BE000290A004C25640A0011241FBECFEFDAE069
:100BF000DEBFCDBF04B603FE28C08091D004909123
:100C0000D104A091D204B091D3048730904BA74077
:100C1000B04BD9F41092D0041092D1041092D204A7
:100C20001092D30414BE0FB6F894A895809160007A
:100C3000886180936000109260000FBE10920108DE
:100C400010920008E0E0F8E3099511E0A0E0B1E0BF
:100C5000E6E5F5E502C005900D92AC39B107D9F78C
:100C600024E0ACE9B1E001C01D92A03DB207E1F77C
:100C70000E9446250C94A92A0C9400000FB680957A
:100C80009AE0F8947BE27A95F1F708F0589A08F424
:100C9000589886959A95B1F70FBE08950FB680E8DB
:100CA000F894499BFECF4999FECF96E19A95F1F7CA
:100CB0009CE29A95F1F7869549998068C8F70FBE2E
:100CC00008950FB680E8F89496E19A95F1F79CE2C2
:100CD0009A95F1F7869549998068C8F796E19A95B3
:100CE000F1F7499BFECF0FBE0895FF93EF93E0917C
:100CF0009C01F0919D01309709F00995EF91FF91CA
:100D00000895FC018591803011F0EFDFFBCF08954D
:100D1000FF27E0E230E247FF0CC0419597FF09C092
:100D2000EDE26095709580959095611D711D811D16
:100D3000911D27FF02C0219530E350E2AA27660FDC
:100D4000771F881F991FAA1FA41710F0A41B639573
:100D50005A95A9F7AA3008F0A95FA05DAF93F39563
:100D6000611571058105910541F7ED3211F4EF939D
:100D7000F395F21718F43F93F395FBCF8F91B5DFFE
:100D8000FA95E1F70895E991F9918591803021F084
:100D9000853219F0AADFF9CF089520E0E894559143
:100DA0005532C1F3503311F4689455915A3348F4D5
:100DB000505390F3220F022E220F220F200D250FE9
:100DC000F4CF0EF4219589919991533619F3533745
:100DD00029F1533559F1BC0188279927E8945C36ED
:100DE00021F48991999168945591543639F446EFDC
:100DF0007EF077FF0DC08FEF9FEF0AC055374AE0B6
:100E000039F0583540E121F0523642E009F00895BA
:100E1000FF93EF937DDFEF91FF91B7CFFF93EF93B8
:100E2000FC0181918030B9F360DFFBCFFF93EF933A
:100E300068DFF1CFDF93CF93CDB7DEB72596A3DF81
:100E4000CF91DF910895803FC1F48091C60487FD62
:100E50001092C6048091C50481110EC08091C60411
:100E600081110AC08091C704811106C08091C80415
:100E7000811102C01092BF040895813F29F480912E
:100E8000C60418162CF3E6CF9091C504823F29F4CE
:100E900097FFE0CF1092C504DDCF833F19F41916F8
:100EA000CCF3D8CF893F39F48091C704181694F653
:100EB0001092C704CFCF8A3F29F48091C70487FFDF
:100EC000C9CFF6CF8B3F39F48091C80487FFC2CFDA
:100ED0001092C804BFCF8C3F29F48091C804181623
:100EE000BCF3B8CF843F31F48091C4048E7F8093EB
:100EF000C404B0CF853F21F48091C4048D7FF7CF27
:100F0000863F21F48091C4048B7FF1CF873F21F489
:100F10008091C404877FEBCF883F21F48091C40483
:100F20008F7EE5CF8D3F31F48091BE048E7F80931C
:100F3000BE0490CF8E3F21F48091BE048D7FF7CF09
:100F40008F3F09F087CF8091BE048B7FF0CF8091D7
:100F5000BE0480FF0CC060912A0170E07595679512
:100F6000759567956115710549F1862F089581FF83
:100F700006C060912A0170E075956795F3CF609186
:100F80002A0182FD0BC09091BF049923A1F06091CA
:100F9000290180912A01961738F0682F70E0603897
:100FA000710500F38FE70895899FC001112470E057
:100FB0000E946D2AF4CF61E070E0D7CF81E0089500
:100FC0008091BE0480FF12C060912C0185E0689F73
:100FD000B001112475956795759567956038710511
:100FE000A8F561157105A1F1862F089581FF09C04B
:100FF00060912C0185E0689FB0011124759567957B
:10100000EDCF82FF07C060912C0185E0689FB001A1
:101010001124E4CF2091BF042223A9F090912B0149
:1010200060912C0185E0689FB00111242917B0F66A
:10103000269FA001279F500D1124692F70E0CA013F
:101040000E946D2ACBCF65E070E0CECF8FE7089588
:1010500081E00895803F31F40E94E00781958093FC
:10106000C6040895813F19F40E94E007F8CF823F3B
:1010700031F40E94E00781958093C5040895833F71
:1010800019F40E94E007F8CF893F29F40E94A707CE
:101090008093C70408958A3F21F40E94A707819591
:1010A000F7CF8B3F31F40E94A70781958093C80446
:1010B00008958C3F19F40E94A707F8CF843F31F4BC
:1010C0008091C40481608093C4040895853F21F415
:1010D0008091C4048260F7CF863F21F48091C404DC
:1010E0008460F1CF873F21F48091C4048860EBCF06
:1010F000883F21F48091C4048061E5CF8D3F31F4B5
:101100008091BE0481608093BE0408958E3F21F4D7
:101110008091BE048260F7CF8F3FB9F78091BE0403
:101120008460F1CF28E0729FF0011124E60FF11DD9
:10113000E95EF94F6491E62FE295E77028E0829F1F
:10114000C00111248E0F911D24E0880F991F2A954C
:10115000E1F7E62FEF70E80FF92FF11DEE0FFF1FFB
:10116000E050F8498591949108952FB7F8946091D3
:10117000BA047091BB048091BC049091BD042FBF50
:1011800008952FB7F8948091BA049091BB04A09170
:10119000BC04B091BD042FBF08958091B804843081
:1011A00021F11092B90488E190E020E40FB6F894A0
:1011B000A895809360000FBE2093600083B7817F65
:1011C000846083BF83B7816083BF7894889583B739
:1011D0008E7F83BF0FB6F894A895809160008861D8
:1011E00080936000109260000FBE08954F925F924E
:1011F0006F927F929F92AF92BF92CF92DF92EF92C7
:10120000FF920F931F93CF93DF9300D000D01F92D4
:10121000CDB7DEB76B837C838D837A018C819D8112
:10122000892B49F08FEFF81204C081E09FEF491736
:1012300019F080E001C081E080FD67C00F2D10E053
:10124000CE2CD12C8B81882309F453C040906F049D
:101250005090700460907104709072048091CC047E
:101260009091CD04A091CE04B091CF04482A592A80
:101270006A2A7B2A2FE1A22EB12C9A2CD301C2011B
:101280000A2C04C0B695A795979587950A94D2F72E
:1012900080FD28C081E0A81AB10878F7912CF801E8
:1012A00093E0EE0FFF1F9A95E1F7ED58FB4FEC0D21
:1012B000FD1D9082B701892D0F900F900F900F9018
:1012C0000F90DF91CF911F910F91FF90EF90DF90E2
:1012D000CF90BF90AF909F907F906F905F904F9016
:1012E0000C949208B7018A2D0E949208019791F2FE
:1012F000D6CFF80183E0EE0FFF1F8A95E1F7ED5896
:10130000FB4FEC0DFD1D9080D5CF90E080E00F905D
:101310000F900F900F900F90DF91CF911F910F9131
:10132000FF90EF90DF90CF90BF90AF909F907F9015
:101330006F905F904F90089541E050E060E070E062
:1013400004C0440F551F661F771F8A95D2F740953A
:1013500050956095709580916F0490917004A09164
:101360007104B091720484239523A623B72380933C
:101370006F0490937004A0937104B0937204089565
:1013800041E050E060E070E004C0440F551F661F6C
:10139000771F8A95D2F780916F0490917004A09185
:1013A0007104B0917204842B952BA62BB72B8093DC
:1013B0006F0490937004A0937104B0937204089525
:1013C00080916E0490913D04981301C008958F5F41
:1013D0008770FACF1F93CF93DF9300D000D01F9276
:1013E000CDB7DEB7942F4983252F5A836B837C8337
:1013F0008D834C815D8181E0452B31F02F3F19F4C5
:1014000081E09F3F09F080E0182F117080FD2CC013
:1014100049815A816B817C818D810E94F608292F38
:1014200022952F702C3078F42A30A8F422502230E4
:10143000C8F0812F0F900F900F900F900F90DF91B9
:10144000CF911F9108952C3011F02F3091F793FB1D
:10145000112710F9EECF803C28F0803E50F3815FD9
:10146000833038F311E0E5CF10E0E3CFE091C00422
:10147000F091C104309721F00190F081E02D0994A2
:1014800080E00895E8EDF0E080818E7F8083109207
:10149000E2001092DA001092E100A0EEB0E08C9130
:1014A00081608C9380818F77808319BCA7EDB0E039
:1014B0008C918E7F8C9380818F7E80831092040428
:1014C00008950E94420AF89487E797E790930108ED
:1014D0008093000887E090EBDC018093D004909328
:1014E000D104A093D204B093D30488E19CE00FB65A
:1014F000F894A895809360000FBE90936000FFCF92
:10150000FC01809130049091310486179707A0F078
:101510006115710529F49091E8009E779093E80099
:1015200090E06115710551F4911108C08091E800B7
:1015300082FF35C080E00895BC01F2CF8091B804ED
:101540008823C9F18530C9F18091E80083FD31C05D
:101550008091E80082FDEACF8091E80080FFE1CF32
:101560002091F3008091F200322F282F6115710530
:1015700019F02830310558F091E02830310509F094
:1015800090E02091E8002E772093E800CACF819167
:101590008093F100615071092F5F3F4FE7CF809139
:1015A000B804882341F0853041F08091E80083FF42
:1015B000BDCF81E0089582E0089583E008952091F1
:1015C000E4003091E50085E69091EC0090FF06C0C4
:1015D0009091E80090FF06C080E008959091E800A7
:1015E00092FDFACF9091B804992391F0953091F043
:1015F0009091EB0095FD10C04091E4005091E50002
:101600002417350709F381509A01F1F684E0089513
:1016100082E0089583E0089581E00895EF92FF92BB
:101620000F931F93CF937C018B010E94DF0AC82F79
:10163000811117C08091E80085FD0BC08091E80002
:101640008E778093E8000E94DF0A882399F3C82FE1
:1016500008C0F70181917F018093F10001501109C9
:1016600049F78C2FCF911F910F91FF90EF90089524
:1016700080912A0487FF13C08091E80082FF06C092
:101680008091E8008B778093E80004C08091B804D3
:101690008111F2CF08958091B8048823D9F3809105
:1016A000E80080FFF8CF8091E8008E77ECCF982F8C
:1016B0009093E900242F762F50E0891731F0709134
:1016C000EC002091ED005091F00021FD07C09F5FDC
:1016D000973071F78093E90081E008953091EB0035
:1016E0003E7F3093EB003091ED003D7F3093ED0075
:1016F0003091EB0031603093EB007093EC0020935D
:10170000ED005093F0002091EE0027FDE0CF80E047
:101710000895CF92DF92EF92FF920F931F93CF9392
:10172000DF93C8EDD0E088818F7E8883E7EDF0E01D
:1017300080818160808384E082BF81E080930404A3
:1017400088818E7F888302EE10E0F801108210926B
:10175000DA0081EEC82ED12CF601108288818F77B5
:10176000888388818068888388818F7D888319BC7D
:101770001092B804109229041092280410922704A1
:1017800090EEE92EF12CF70180818B7F8083888198
:101790008160888342E060E080E00E94570BF601A0
:1017A00080818E7F8083F801808181608083808149
:1017B00088608083F70180818E7F8083888180614B
:1017C0008883DF91CF911F910F91FF90EF90DF9071
:1017D000CF9008958091060408950895089508957E
:1017E000089508958091FD0308958091FD03089563
:1017F000879A8F9A08959091C80095FFFCCF8093A7
:10180000CE000895CF93DF938D3C910509F451C02C
:1018100090F5D0E0C1E0853B9105E1F060F4D0E0C7
:10182000C0E1833B9105B1F0D0E0C0E2843B91057B
:1018300089F0D0E02DC0D0E0C4E0873B910551F0A5
:10184000D0E0C2E0873B910528F0D0E0C8E08C3CB6
:10185000910579F78DEF0E94FB0B83E00E94FB0B53
:1018600083E00E94FB0B8D2F0E94FB0B8C2FDF91DE
:10187000CF910C94FB0BD0E28A3E910549F050F4D5
:10188000D0E4823E910521F0D0E1893E910589F6B0
:10189000C0E0E0CFD4E0813222E09207C9F3D1E08A
:1018A000833222E09207A1F3D2E08A38914009F610
:1018B000EFCFD0E8EDCFCF93DF93EC018DEF0E9417
:1018C000FB0B85E00E94FB0B82E00E94FB0B8881F2
:1018D0000E94FB0B89810E94FB0B8A810E94FB0BFB
:1018E0008B81DF91CF910C94FB0BCF93DF93EC01B5
:1018F0008DEF0E94FB0B89E00E94FB0B81E00E94B0
:10190000FB0B88810E94FB0B80E00E94FB0B8A810D
:101910000E94FB0B8B810E94FB0B8C810E94FB0BB6
:101920008D810E94FB0B8E810E94FB0B8F81DF91CA
:10193000CF910C94FB0B4091C3039091C2034917C4
:10194000D1F0292F30E0F901EE53FD4F80812F5F58
:101950003F4F33279F5F9093C203642F70E0261B95
:10196000370B491730F4233031050CF05D9890E0C7
:1019700008953395F8CF8FEF9FEF089514B88FEF48
:1019800085B9549A5C9808950C94BE0C8330C9F1C3
:1019900028F4813061F0823019F10895853009F41E
:1019A00052C008F43FC0863009F45EC008958091AB
:1019B0002E01681790F4861B80932E0180912E01D2
:1019C0001F928F938BE89AE09F938F930E941A0740
:1019D0000F900F900F900F90089510922E01EECF60
:1019E00080912D01681750F4861B80932D01809102
:1019F0002D011F928F9389E79AE0E6CF10922D0177
:101A0000F6CF80912C01681750F4861B80932C012F
:101A100080912C011F928F9386E69AE0D5CF109289
:101A20002C01F6CF80912B01681750F4861B809310
:101A30002B0180912B011F928F9381E59AE0C4CFF7
:101A400010922B01F6CF80912A01681750F4861B63
:101A500080932A0180912A011F928F9388E39AE054
:101A6000B3CF10922A01F6CF80912901681750F464
:101A7000861B80932901809129011F928F938DE10C
:101A80009AE0A2CF10922901F6CF833009F445C025
:101A900028F4813061F0823049F10895853009F4ED
:101AA0006AC008F451C0863009F47CC00895809162
:101AB0002E01482F460F5527551F4F3F510594F4CF
:101AC000680F60932E0180912E011F928F938EE0FC
:101AD0009AE09F938F930E941A070F900F900F9098
:101AE0000F9008958FEF80932E01EDCF80912D01FF
:101AF000482F460F5527551F4F3F510554F4680F87
:101B000060932D0180912D011F928F938CEF99E0AE
:101B1000E0CF8FEF80932D01F5CF80912C01482FDE
:101B2000460F5527551F4F3F510554F4680F6093DA
:101B30002C0180912C011F928F9389EE99E0C9CFDF
:101B40008FEF80932C01F5CF80912B01482F460F0A
:101B50005527551F4F3F510554F4680F60932B01D3
:101B600080912B011F928F9384ED99E0B2CF8FEF7C
:101B700080932B01F5CF80912A01482F460F5527DE
:101B8000551F4F3F510554F4680F60932A0180910F
:101B90002A011F928F938BEB99E09BCF8FEF80935D
:101BA0002A01F5CF80912901482F460F5527551F4F
:101BB0004F3F510554F4680F60932901809129012A
:101BC0001F928F9380EA99E084CF8FEF8093290151
:101BD000F5CFCF93DF93209134043091350428174B
:101BE000390701F19093350480933404E091C004E7
:101BF000F091C1043097B1F0EC010084F185E02D43
:101C000009958091CB048570853061F4DF93CF9383
:101C10008AE295E09F938F930E941A070F900F908E
:101C20000F900F90DF91CF910895CF93DF93209184
:101C30003204309133042817390701F190933304AB
:101C400080933204E091C004F091C1043097B1F068
:101C5000EC010680F781E02D09958091CB04857019
:101C6000853061F4DF93CF938CE195E09F938F9360
:101C70000E941A070F900F900F900F90DF91CF9155
:101C80000895CF93DF93CBE8D1E00E949B0C8F3F68
:101C9000980719F4DF91CF9108959F938F93DF9365
:101CA000CF930E941A070F900F900F900F90EDCFD7
:101CB00088EE9AE00E9481061F9281E08F931F9226
:101CC00085E08F938AE99AE09F938F930E941A0789
:101CD0000F900F900F900F900F900F900895CF934B
:101CE0008091CB0483FF7EC08EE796E00E94810640
:101CF0008091C4041F928F9389E796E09F938F93FE
:101D00000E941A0787E796E00E9481068091C50429
:101D1000282F082E000C330B3F938F9384E796E017
:101D20009F938F930E941A0782E796E00E94810694
:101D30008091C604282F082E000C330B3F938F93FD
:101D40008FE696E09F938F930E941A078DE696E0A8
:101D50000E9481068091C704282F082E000C330BA7
:101D60003F938F938AE696E09F938F930E941A0782
:101D700088E696E00E9481068091C804282F082EEC
:101D8000000C330B3F938F9385E696E09F938F93E0
:101D90000E941A0782E696E00E9481068091BF04A5
:101DA0001F928F938FE596E09F938F930E941A075F
:101DB0008DE596E00E9481068091BE041F928F936C
:101DC0008AE596E09F938F930E941A0787E596E035
:101DD0000E9481068DB79EB74C960FB6F8949EBFB1
:101DE0000FBE8DBFE091C004F091C1043097F1F1B6
:101DF000C091C4040480F581E02D84EC94E0099541
:101E0000C093C4048091CB0483FF30C08091C80488
:101E1000282F082E000C330B3F938F938091C7041B
:101E2000282F082E000C330B3F938F938091C6040C
:101E3000282F082E000C330B3F938F938091C504FD
:101E4000282F082E000C330B3F938F931F92CF93B4
:101E500081EA96E09F938F930E941A078DB79EB7F1
:101E60000C960FB6F8949EBF0FBE8DBF0E94C1089E
:101E70009093C3048093C204CF9108950F931F934E
:101E8000CF93DF938091B7049091B604892B809310
:101E90009E028091B5048823B1F10E94C10820916F
:101EA000B3043091B404821B930B8C32914090F0B8
:101EB0008091CB0480FF08C085E096E09F938F93CC
:101EC0000E941A070F900F901092B5041092B4045C
:101ED0001092B30480919E029091B504892B809357
:101EE0009E02EFE9F2E080E0919191118F5F92E024
:101EF000EE3BF907C9F7882331F01092B504109230
:101F0000B4041092B304E091C004F091C10430977E
:101F1000B1F10280F381E02D8EE992E00995809184
:101F2000CB0482FF2CC080FF04C08AEF95E00E94A2
:101F30008106D0E0C0E004EF15E08091CB0480FF83
:101F40000EC0FE01E256FD4F80811F928F931F93BA
:101F50000F930E941A070F900F900F900F902196E9
:101F6000C032D10551F78091CB0480FF08C082EFC9
:101F700095E0DF91CF911F910F910C948106DF9135
:101F8000CF911F910F9108951092B7041092B6044B
:101F9000EFE9F2E0119282E0EE3BF807D9F70E94F8
:101FA0003E0F85E0E4ECF4E0DF011D928A95E9F74D
:101FB0001092BF041092BE040E946F0E90E080E069
:101FC0000E94150E90E080E00C94E90DCF93C82F8D
:101FD0001F928F9383EE9BE09F938F930E941A072B
:101FE00081E090E0A0E0B0E004C0880F991FAA1F34
:101FF000BB1FCA95D2F78093CC049093CD04A093D5
:10200000CE04B093CF040F900F900F900F90CF910C
:102010000C94C40F882341F080959091B7048923D4
:102020008093B7040C943E0F0895882339F0909163
:10203000B704892B8093B7040C943E0F089588232E
:1020400009F45BC09CEF980F913A60F590912801DC
:102050009923D9F0909127019923B9F0E82FE695BB
:10206000E695E695F0E0E256FD4F877021E030E01E
:10207000A90102C0440F551F8A95E2F7CA01809555
:102080009181892381830C943E0FEEE9F2E02CEBE1
:1020900032E09281891301C0128231962E173F07D8
:1020A000C1F7F1CF90E2980F983088F4877021E063
:1020B00030E0A90102C0440F551F8A95E2F7CA011A
:1020C00080959091B70489238093B704DCCF9BE57A
:1020D000980F933020F490E080E00C94150E98E572
:1020E000980F973120F490E080E00C94E90D803F48
:1020F00020F00E9423070C946F0E0895CF9387322F
:1021000008F050C08E3108F017C1803109F4A9C021
:10211000F8F4873009F488C048F4863009F471C0B7
:102120008EE797E00E948106C0E027C08B3009F45B
:1021300063C08E30A9F79091CB04892F8B7F92FFDB
:1021400084608093CB0482FF89C088E499E07DC0DD
:10215000863109F4ADC0A0F4813111F70E94C40F9B
:10216000C091270181E0C827C0932701CC2309F43F
:10217000E0C08BE897E00E9481068C2FCF910895F4
:10218000893109F47EC08B3159F69091CB04892FA7
:102190008D7F91FF82608093CB0481FF5CC085E6D8
:1021A00099E053C0883341F158F4893229F08533DE
:1021B00019F0873209F0B4CF80E00E94E60F32C0F8
:1021C0008334D1F328F48A3308F4AACF8953F5CFA6
:1021D000883409F0A5CF0E94C40F8BE899E00E94D3
:1021E00081062FEF83ED90E3215080409040E1F78E
:1021F00000C000000E94610A8CEB96E00E948106FC
:1022000011C08091CB04817F8E7F8093CB0487E5C2
:1022100097E00E9481068CE999E00E94810681E0A6
:102220008093CA04C1E0A9CF8091CB0480FF0BC08A
:102230008EE799E00E9481068091CB04817F8E7F9A
:102240008093CB04EFCF82E799E00E9481068091D2
:10225000CB048160F5CF87E599E0D0CF88E399E0A2
:10226000CDCF9091CB04892F877F93FF8860809397
:10227000CB0483FF03C08CE299E0E7CF8FE199E0C4
:10228000BDCF80E199E00E94810683EE98E00E9434
:1022900081068CEA98E00E94810686E898E00E9418
:1022A00081068CE398E00E94810681E198E0A6CF48
:1022B00083E098E00E9481060E94360A1F928F9365
:1022C00089EE97E09F938F930E941A0780912801CF
:1022D0001F928F9382ED97E09F938F930E941A072E
:1022E0008091C9041F928F938FEB97E09F938F93F8
:1022F0000E941A07809127011F928F938CEA97E022
:102300009F938F930E941A070E94B5089F938F9303
:102310007F936F9385E997E09F938F930E941A07AD
:102320008DB79EB746960FB6F8949EBF0FBE8DBF71
:1023300079CF80E897E062CF8D513FCFCF93DF9385
:1023400000D01F92CDB7DEB72091B804243041F5FC
:1023500020912601222321F123E029839B838A8374
:1023600082E08093E9008FEF9091E800815095FD25
:1023700006C095ED9A95F1F700008111F5CF809197
:10238000E80085FF0DC050E040E063E070E0CE0162
:1023900001960E940E0B8091E8008E778093E800F2
:1023A0000F900F900F90DF91CF910895CF93DF930F
:1023B00000D01F92CDB7DEB72091B804243081F54C
:1023C00020912601222361F119821A821B8222E0C8
:1023D00029838138910520F0805891099B838A8355
:1023E00082E08093E9008FEF9091E800815095FDA5
:1023F00006C095ED9A95F1F700008111F5CF809117
:10240000E80085FF0DC050E040E063E070E0CE01E1
:1024100001960E940E0B8091E8008E778093E80071
:102420000F900F900F90DF91CF9108952091B804F5
:10243000243049F522E02093E9002FEF3091E800A5
:10244000215035FD06C035ED3A95F1F70000211118
:10245000F5CF2091E80025FF16C02091260150E01D
:1024600040E063E070E0222339F021E02093F100A6
:1024700050E040E065E070E00E940E0B8091E800C3
:102480008E778093E8000895CF93DF932091B8046E
:102490002430D9F4EC01809128018823F1F0809157
:1024A00027018823D1F081E08093E90081E8815001
:1024B00021F09091E80095FF0BC08091E80050E07A
:1024C00040E060E270E085FD1AC0DF91CF91089591
:1024D0009AE29A95F1F700C0EACF81E08093E90093
:1024E00081E8815021F09091E80095FF19C080911A
:1024F000E80085FFEACF50E040E068E070E0CE0100
:102500000E940E0B8091E8008E778093E80080E2B5
:10251000FE01A7E0B4E001900D928A95E1F7D5CFD6
:10252000EFE3F1E03197F1F700C00000DACFCF938D
:10253000DF9300D0CDB7DEB7849A8C9A80917A0071
:10254000806880937A008FE99FE00197F1F700C0DF
:10255000000080917A00806480937A0080917A00F4
:1025600086FDFCCF80917800909179009A838983D1
:1025700080917A008F7780937A00849A8C98298151
:102580003A8145E0429FC001439F900D1124805540
:1025900091090F900F90DF91CF9108958091D9000C
:1025A00080FF21C08091D90080FF1BC090B331B360
:1025B00085988D9AEFE9FFE03197F1F700C00000B0
:1025C0008FB185FB882780F921E0822720B32F7DFA
:1025D0009072292B20BB91B39F7D3072932B91BBBE
:1025E000089580E008950E9497128C3AFDE09F07BD
:1025F00048F481E08093DE038091DE03811108C0FE
:1026000082E0089585379E40B8F31092DE03F4CF40
:1026100083E008950F931F93CF938C01F801C49129
:102620000F5F1F4FC1114EC0FFEF29E688E1F15047
:1026300020408040E1F700C000000E94C1088C01EA
:102640002FB7F8948091BA049091BB04A091BC0478
:10265000B091BD042FBF801B910B8436910588F487
:102660000E949B0C8F3F980751F08D3041F08A30CB
:1026700041F0EC2FF0E0EC53FC4F8083CF5FC7318B
:10268000F9F684EC93E0EC2FF0E0EC53FC4F108271
:102690009093DD038093DC039F938F9386E891E012
:1026A0009F938F930E941A070E94410E0F900F90E4
:1026B0000F900F908091DC039091DD03CF911F91DB
:1026C0000F9108958C2F0E94FB0BA8CF8AEB91E00D
:1026D0000E94810684EB91E00E940A130E94F80B8D
:1026E0000E94C40F80910A0190910B019093C10444
:1026F0008093C00408958091C0049091C104909388
:102700000B0180930A010E94C40F80E091E0909336
:10271000C1048093C004879A8F987E99FECF8AE97E
:1027200091E00E9481062FEF85EB95E321508040D8
:102730009040E1F700C0000086E991E00E940A1392
:10274000EFEFFBE42DE1E150F0402040E1F700C065
:1027500000000E94410E82E991E00E940A13FC01F0
:102760008081863721F08EE891E00C940A13089559
:102770004F925F926F927F928F929F92AF92BF9291
:10278000CF92DF92EF92FF92CF93833109F474C01E
:10279000D0F48B3009F43FC030F4853009F4A4C183
:1027A000C09102045AC08C3009F473C08131C1F762
:1027B000C1E08091C0049091C1048251914009F020
:1027C0004CC0C0E04AC0883331F190F4883141F701
:1027D000809102048111F5CFC0910104CC2309F44A
:1027E000E0C182E492E00E9481061092010435C0AB
:1027F000873409F4E5C18C3499F6C1B3CC1FCC27DA
:10280000CC1F09F4D6C10E947B1381E08093CA04D7
:102810008093020422C08CEE93E00E94810687ED33
:1028200093E00E9481068DEB93E00E94810686E989
:1028300093E00E9481068BE793E00E94810689E67F
:1028400093E00E948106C0910204CC2311F0C1E004
:1028500004C089E493E00E9481068C2FCF91FF9001
:10286000EF90DF90CF90BF90AF909F908F907F9030
:102870006F905F904F9008950E947B1389ED91E0D7
:102880000E940A1383ED91E00E940A130E946613CE
:10289000DECF80E393E00E9481068091C004909196
:1028A000C1048C51914009F48EC085E391E09F935F
:1028B0008F9382E293E09F938F930E941A078091F7
:1028C00001041F928F9383E193E09F938F930E9463
:1028D0001A078DB79EB708960FB6F8949EBF0FBE25
:1028E0008DBF799973C07E9974C083E491E09F9302
:1028F0008F9389E093E09F938F930E941A0781B38F
:10290000082E000C990B892F881F8827881F1F927B
:102910008F938EEE92E09F938F930E941A0780917F
:1029200002041F928F938DED92E09F938F930E94EC
:102930001A078091B8042DB73EB7245F3F4F0FB6FA
:10294000F8943EBF0FBE2DBF882309F445C0809187
:10295000B804813009F443C08091B804823009F48E
:1029600041C08091B804833009F43FC08091B8041D
:102970008430F1F18091B8048530E9F180E891E08C
:102980009F938F938EEC92E09F938F930E941A07F0
:1029900084EC92E09F938F930E941A070E94CE12BC
:1029A0000F900F900F900F900F900F90813009F4BF
:1029B00092C020F1823009F491C0833009F491C0B3
:1029C0008CEA92E01DC08FE291E071CF8AE391E042
:1029D0008ECF8EE391E08BCF86E491E0D1CF81E57D
:1029E00091E0CECF89E591E0CBCF81E691E0C8CFF1
:1029F0008BE691E0C5CF86E791E0C2CF8FEB92E006
:102A00009F938F930E941A070F900F908AEA92E08B
:102A10009F938F930E941A07809128041F928F938F
:102A200081E992E09F938F930E941A078091D900C9
:102A300081701F928F9387E892E09F938F930E94FB
:102A40001A070E94B5086B017C0128EE33E040E0D4
:102A500050E00E94812A29013A013CE3832E912C07
:102A6000A12CB12CC301B201A50194010E94812ABD
:102A70007F936F93C301B20120E13EE040E050E05C
:102A80000E94812AA50194010E94812A3F932F93DD
:102A9000C701B60120E83EEE46E350E00E94812ADD
:102AA0001F922F93C701B60120E03CE546E255E0B6
:102AB0000E94812A3F932F938AE692E09F938F93FF
:102AC0000E941A078DB79EB744960FB6F8949EBF22
:102AD0000FBE8DBFBCCE89EB92E092CF82EB92E02D
:102AE0008FCF8EEA92E08CCF0E94B5086B017C01FB
:102AF00028EE33E040E050E00E94812A49015A016B
:102B00000E9497129F938F938FE592E09F938F93EC
:102B10000E941A07C701B60120E83EEE46E350E0E6
:102B20000E94812A5F934F933F932F9389E592E010
:102B30009F938F930E941A07C501B40120E13EE0E4
:102B400040E050E00E94812A2CE3C22ED12CE12CDF
:102B5000F12CA70196010E94812A5F934F933F9326
:102B60002F9383E592E09F938F930E941A07C501EC
:102B7000B401A70196010E94812A9F938F937F93AE
:102B80006F938DE492E09F938F930E941A072DB765
:102B90003EB72A5E3F4F0FB6F8943EBF0FBE2DBF23
:102BA00056CE88E392E00E94810681E08093010482
:102BB0004ECE0E9466131092CA041092020447CEB1
:102BC00080910204811102C00E947B1381E392E094
:102BD0000E940A1386E292E00E940A1382E192E0C8
:102BE0000E940A138BE092E00E940A1381E092E0B7
:102BF0000E940A138AEF91E00E940A1380EF91E08D
:102C00000E940A1386EE91E00E940A1380EE91E082
:102C10000E940A1380910204811119CE37CECF93FE
:102C2000DF93C82F882309F4FFC1ECEFE80FE13AE6
:102C300008F0C0C28091CA048130A9F130F082301E
:102C400009F4A9C11092CA040FC080919E02823279
:102C500059F48C2F0E94B81381117DC08C2F0E94D3
:102C60007E10817009F0E0C180912801882309F469
:102C700087C280912701882309F482C2EC2FE69550
:102C8000E695E695F0E0E256FD4FC77021E030E0B2
:102C900001C0220FCA95EAF78181822B8183DF91DF
:102CA000CF910C943E0F80919E02823291F28091DE
:102CB000B7048272E93408F027C1F0E0EE59F94E0A
:102CC0000C94A32AB416B916BE16C316C816CD1690
:102CD000D216D716DC16E116E616EB16F016F61627
:102CE000FC16021708170E1714171A1720172617A5
:102CF0002C17321738173E1744174A175017561714
:102D00005C17621768176E1774177A17C917AE1613
:102D100080178217841786178B17911797179D179F
:102D20009D17A317A917AF17B517BB17C11784179E
:102D300084178417841784178417841784178417BB
:102D400084178417841784178417841784178417AB
:102D500084178417C71781E090E083CFCBE18C2FD5
:102D6000DF91CF910C94FB0BC1E68823C1F3C1E442
:102D7000F6CFC2E6882399F3C2E4F1CFC3E68823F5
:102D800071F3C3E4ECCFC4E6882349F3C4E4E7CF8E
:102D9000C5E6882321F3C5E4E2CFC6E68823F9F22D
:102DA000C6E4DDCFC7E68823D1F2C7E4D8CFC8E6B2
:102DB0008823A9F2C8E4D3CFC9E6882381F2C9E405
:102DC000CECFCAE6882359F2CAE4C9CFCBE688231E
:102DD00031F2CBE4C4CFCCE6882309F2CCE4BFCFF8
:102DE000CDE6882309F4BBCFCDE4B9CFCEE6882366
:102DF00009F4B5CFCEE4B3CFCFE6882309F4AFCF43
:102E0000CFE4ADCFC0E7882309F4A9CFC0E5A7CFB1
:102E1000C1E7882309F4A3CFC1E5A1CFC2E7882386
:102E200009F49DCFC2E59BCFC3E7882309F497CF70
:102E3000C3E595CFC4E7882309F491CFC4E58FCFCC
:102E4000C5E7882309F48BCFC5E589CFC6E788237A
:102E500009F485CFC6E583CFC7E7882309F47FCF80
:102E6000C7E57DCFC8E7882309F479CFC8E577CFD8
:102E7000C9E7882309F473CFC9E571CFCAE788236E
:102E800009F46DCFCAE56BCFC1E3882309F467CF9E
:102E9000C1E265CFC2E3882309F461CFC0E45FCF0C
:102EA000C3E3882309F45BCFC3E259CFC4E388238B
:102EB00009F455CFC4E253CFC5E3882309F44FCFBB
:102EC000C5E24DCFC6E3882309F449CFCEE547CF0D
:102ED000C7E3882309F443CFC6E241CFC8E3882380
:102EE00009F43DCFCAE23BCFC9E3882309F437CFC9
:102EF000C8E235CFC0E3882309F431CFC9E22FCF30
:102F0000C8E02DCFC9E02BCFC0E229CF882309F438
:102F100026CFCFE524CFCDE3882309F420CFCBE221
:102F20001ECFCBE5882309F41ACFCBE718CFCDE528
:102F3000882309F414CFCDE712CFCCE5882309F418
:102F40000ECFCCE70CCFCBE3882309F408CFCAE33C
:102F500006CFC7E2882309F402CFC2E200CFC0E661
:102F6000882309F4FCCECEE7FACECCE2882309F41C
:102F7000F6CECCE3F4CECEE2882309F4F0CECEE355
:102F8000EECECFE2882309F4EACECFE3E8CEC0E06C
:102F9000E6CECAE0E4CEC432D0F4CE3108F0C0C0F0
:102FA000CB30E9F048F4C73009F4D0C08FED95E09C
:102FB000DF91CF910C948106C331C9F1C431B1F7CF
:102FC00080913604882349F1109236040AC0CB342C
:102FD00009F4BAC0C0F4C93299F3C83339F70E9472
:102FE000580E80913604882309F4C7C01F928F932E
:102FF00089ED95E09F938F930E941A070F900F9091
:103000000F900F9011C0C13509F498C0C23509F472
:103010008FC0CE3459F66AE092C08EEE95E00E94E1
:10302000810681E08093CA04DF91CF91089588ECF6
:1030300095E00E94810686EB95E00E9481068091D2
:103040002E011F928F9383EB95E09F938F930E94A5
:103050001A0781EB95E00E9481068FE995E00E94B6
:10306000810680912D011F928F938CE995E09F93AB
:103070008F930E941A078AE995E00E9481068BE8E7
:1030800095E00E94810680912C011F928F9388E821
:1030900095E09F938F930E941A0786E895E00E941F
:1030A000810685E795E00E94810680912B011F92A1
:1030B0008F9382E795E09F938F930E941A0780E792
:1030C00095E00E9481068BE595E00E948106809143
:1030D0002A011F928F9388E595E09F938F930E941A
:1030E0001A0786E595E00E9481068FE395E00E942D
:1030F0008106809129011F928F938CE395E09F9325
:103100008F930E941A078AE395E00E9481068DB78B
:103110009EB748960FB6F8949EBF0FBE8DBF61CF85
:10312000CE51D0E0CF56DE4F88818093360459CF00
:1031300061E0809136040E94450D53CF61E080919B
:1031400036040E94C60C4DCF6AE0F3CF8EE1809327
:103150002E0182E380932D018AE080932C0184E18B
:1031600080932B0188E080932A0188E280932901D3
:1031700081EE95E00E94810634CF86ED95E018CF70
:10318000A0EAB2E0EFEF80E09D91C91709F487CD86
:10319000EF3F19F4911101C0E82F8F5F8E31A1F735
:1031A000EF3F09F47CCD0E2E000CFF0BE256FD4FD5
:1031B000C28375CD80E28C0F883068F4C77021E03F
:1031C00030E001C0220FCA95EAF78091B704822B44
:1031D0008093B70464CD8BE58C0F833070F481E865
:1031E00090E0C53A31F083E890E0C63A11F482E805
:1031F00090E0DF91CF910C94150E88E58C0F87310C
:1032000008F069C082EE90E0C83A09F460C089EE27
:1032100090E0C93A09F45BC08AEE90E0CA3A09F43A
:1032200056C085EB90E0CB3A09F451C086EB90E0B4
:10323000CC3A09F44CC083EB90E0CD3A09F447C096
:1032400084EB90E0CE3A09F442C087EB90E0CF3AAD
:10325000F1F188EB90E0C13BD1F18DEC90E0C03B07
:10326000B1F183E891E0C23B91F18AE891E0C33B80
:1032700071F182E991E0C43B51F184E991E0C53BF1
:1032800031F181E292E0C63B11F183E292E0C73B6B
:10329000F1F084E292E0C83BD1F085E292E0C93BD4
:1032A000B1F086E292E0CA3B91F087E292E0CB3B3C
:1032B00071F08AE292E0CC3B51F08FE690E0CD3B9A
:1032C00031F090E080E0CE3B11F480E790E0DF91B8
:1032D000CF910C94E90DCF3B69F40E94C40F9FEF8E
:1032E00020E782E0915020408040E1F700C00000DC
:1032F0000E94610AC03F08F497CE8C2F0E942A08D2
:10330000DF91CF910C946F0ECF92DF92EF92FF92EC
:103310000F931F93CF93DF9300D000D01F92CDB7B0
:10332000DEB76C0185E0F601DE01119601900D9289
:103330008A95E1F7F601408151812381348191E042
:103340002115310531F05F3F19F491E04F3F09F04D
:1033500090E090FD9FC0F6010281F580F2949FE01D
:10336000F92249835A830B83722F3D832C83602F6C
:103370008D810E94F608182FE92FE295EF70EF304B
:1033800008F088C0F0E0E953F64E0C94A32AD61951
:10339000D619141A141A941AC61A4A1A4A1ADC1A96
:1033A0004A1AB21BB21B4A1A4A1A6E1CF92FFF7036
:1033B000FF2E907F19F0F29480EFF8220023C9F0DD
:1033C000FF2039F08091B604F82AF092B6040E94EA
:1033D0003E0F812F0F900F900F900F900F90DF9165
:1033E000CF911F910F91FF90EF90DF90CF900C94B1
:1033F0000F16812F0E941F10FF2009F44BC0F0947C
:103400008091B604F822F092B6040F900F900F90BE
:103410000F900F90DF91CF911F910F91FF90EF9040
:10342000DF90CF900C943E0F892F8F70907F903259
:1034300011F08295807F112379F0113009F453C087
:10344000002309F45FC0FF2059F0F601958190FF39
:1034500097C19F70958304C0002351F1F1100FC0F4
:103460000F900F900F900F900F90DF91CF911F91C1
:103470000F91FF90EF90DF90CF900C94151021E00A
:10348000F212EECF8093B5040E94C1089093B40469
:103490008093B3040F900F900F900F900F90DF91D7
:1034A000CF911F910F91FF90EF90DF90CF900895F3
:1034B000F11015C01092B5041092B4041092B30428
:1034C0000F900F900F900F900F90DF91CF911F9161
:1034D0000F91FF90EF90DF90CF900C940A1091E045
:1034E000F912E8CFD7CF002349F0E5E0EF1590F2CD
:1034F0009091B704982309F4B3CFE2CFF4E0FF151D
:1035000048F2DECFFF20E1F2812F0F900F900F9055
:103510000F900F90DF91CF911F910F91FF90EF903F
:10352000DF90CF900C941F10892F8695869583701D
:10353000C1F0813009F0AECF812F9370011102C02C
:1035400090E080E00F900F900F900F900F90DF9120
:10355000CF911F910F91FF90EF90DF90CF900C943F
:10356000E90D812F9370011102C090E080E00F906F
:103570000F900F900F900F90DF91CF911F910F91AF
:10358000FF90EF90DF90CF900C94150E002389F000
:103590000E942A080F900F900F900F900F90DF91CC
:1035A000CF911F910F91FF90EF90DF90CF900C94EF
:1035B0006F0E0E942307EECF892F837009F064C03D
:1035C000011168CF812F829586958770880F880FAB
:1035D000412F4F70C42ED12CF12CE12C082E04C0A9
:1035E000CC0CDD1CEE1CFF1C0A94D2F740E050E02E
:1035F000BA0114FF11C00FE010E020E030E004C079
:10360000000F111F221F331F8A95D2F7B901A8019D
:1036100040955095609570950091CC041091CD0423
:103620002091CE043091CF04969596959370923068
:10363000E9F028F5913089F04C295D296E297F2920
:1036400040235123622373234093CC045093CD0431
:103650006093CE047093CF041DCFC02AD12AE22AF2
:10366000F32A4C295D296E297F29EECF4C295D294B
:103670006E297F294027512762277327E5CF4023F2
:10368000512362237323EDCF8695002311F0892FF8
:103690008170882309F4FECE812F829586958770EC
:1036A000880F880F412F4F70C42ED12CF12CE12CA4
:1036B000082E04C0CC0CDD1CEE1CFF1C0A94D2F7B3
:1036C00040E050E0BA0114FF11C00FE010E020E02C
:1036D00030E004C0000F111F221F331F8A95D2F75C
:1036E000B901A801409550956095709500916F04BF
:1036F0001091700420917104309172049695969502
:1037000093709230E9F028F5913089F04C295D29C9
:103710006E297F29402351236223732340936F0432
:10372000509370046093710470937204B3CE0C29AB
:103730001D292E293F29402B512B622B732BEECFB5
:103740004C295D296E297F2940275127622773273D
:10375000E5CF40235123622373234C295D296E2931
:103760007F29DCCF803F09F44EC0D0F480E4810F84
:10377000803270F1002309F4ACC0FF2009F4A6C028
:10378000812F0E940F16193309F099C0FFEF21EE27
:1037900084E0F15020408040E1F700C000007ACE84
:1037A000823F09F470C008F45BC0833F19F700231F
:1037B00009F47CC0292F2F7181E090E0A0E0B0E0F7
:1037C00004C0880F991FAA1FBB1F2A95D2F73AC0C1
:1037D000E12FE071FE2E892F8F71002351F00E949E
:1037E000C009812F8295807FF1103ACE812F8F7092
:1037F00037CE0E949C09812F8295807FF11060CE88
:10380000812F8F705DCE002331F1F4E0FF1508F4B5
:1038100041CE292F2F7181E090E0A0E0B0E004C0FC
:10382000880F991FAA1FBB1F2A95D2F740916F04DA
:1038300050917004609171047091720484279527EF
:10384000A627B72780936F0490937004A093710408
:10385000B09372041FCE25E02F1508F41BCED9CFEC
:10386000892F8F71002399F00F900F900F900F9078
:103870000F90DF91CF911F910F91FF90EF90DF900C
:10388000CF900C94C009892F8F71002369F30F909A
:103890000F900F900F900F90DF91CF911F910F918C
:1038A000FF90EF90DF90CF900C949C0910926F04E2
:1038B000109270041092710410927204EBCD1335C3
:1038C00009F464CF173409F0E5CD60CF892F8F71EB
:1038D000CBCFF11019CE892F8F71D9CF8111DACDCD
:1038E000002309F4D7CD0E94C40F8FEF90E7E2E0E8
:1038F00081509040E040E1F700C000000E94610A62
:103900000F931F93CF93DF9380913C04807FB9F492
:1039100080913904882399F080916E0410913D04C0
:103920006091370470913804C0913A04D0913B04FF
:1039300021E06F3F09F020E006E0181305C0DF9199
:10394000CF911F910F91089531E0209721F0322FF0
:103950007F3F09F030E090E030FD33C0089FF00178
:10396000099FF00D1124DF01A25CBB4F11963C9121
:103970001197371326C03C91361323C012963C9101
:10398000129731111EC013964D915C914C1B5D0B2B
:103990004C325140B0F480913C048F708061809330
:1039A0003C04ED5BFB4F80818F708061808387E3F7
:1039B00094E00E948419DF91CF911F910F910C9494
:1039C000E00901968770B9CF9F92AF92BF92CF92D4
:1039D000DF92EF92FF920F931F93CF93DF93CDB7B8
:1039E000DEB761970FB6F894DEBF0FBECDBF8C0176
:1039F00085E0F801DE011D9601900D928A95E1F7B0
:103A0000F80140815181F280C380D48090913704C5
:103A10006091380420913A0430913B0481E02115F3
:103A2000310531F06F3F19F481E09F3F09F080E0EC
:103A3000F82FF1709F2E80FD4AC187E3A82E84E005
:103A4000B82EE0903904F601E21BF30B9F01EE2043
:103A500009F400C180913C04782F707F2C323140F2
:103A600008F0BAC0711181C0EF2C651322C0941305
:103A700020C0F1101EC08F70806180933C04C5018E
:103A80000E94841980913C04F80185838E2D6196F3
:103A90000FB6F894DEBF0FBECDBFDF91CF911F915F
:103AA0000F91FF90EF90DF90CF90BF90AF909F90DD
:103AB000089581E0C114D10431F05F3F19F481E031
:103AC0004F3F09F080E080FD24C081E08F25F82F72
:103AD000F170BF2E80FF3FC080916E0420913D04A5
:103AE00036E0821318C07C2DD98AC88A6F2D898947
:103AF0000E94F608292F22952F70223000F12430E1
:103B000028F59F7001F1F8019581907FE1F4E92C8F
:103B1000BDCF80E0DCCF90E0389FF001399FF00D01
:103B20001124E25CFB4F6181561306C0608146138D
:103B300003C062816F110FC001968770D2CF9F7052
:103B400011F0882321F3805E883008F3C8010E94B9
:103B500084199B2CDCCFFF2009F498CF80913C0482
:103B6000816080933C04E12C91CF651306C09413CF
:103B700004C0F801FF2009F488C04D875E87FF86E6
:103B80007C2DD98AC88A6F2D89890E94EA098823E9
:103B900009F4ABC0FF2009F4A8C080913C04803236
:103BA00070F0209137043091380438872F831986BC
:103BB000DB86CA868C87CE0107960E94841986E030
:103BC000F801A7E3B4E001900D928A95E1F70E9415
:103BD000801CEE24E3945ACF71110AC087E394E06D
:103BE0000E94841986E0F50111928A95E9F7BBCF0E
:103BF00065130FC094130DC0F1100BC0F80185833D
:103C0000C8010E94841986E0F50111928A95E9F7AE
:103C10003DCF4D875E87FF867C2DD98AC88A6F2D60
:103C200089890E94EA09882309F45FC0FF2009F40A
:103C30005CC080913C04803210F2209137043091B6
:103C400038043A8329831B82DD82CC828E83CE01A5
:103C50000196B3CF2C323140B0F6EF2CFF2009F49F
:103C600044C065131FC094131DC080913C0480FDA7
:103C700010C0982F907F69F0F8018583903F31F054
:103C8000982F907F905F8F70892B8583C8010E9449
:103C9000841986E0F801A7E3B4E001900D928A95BB
:103CA000E1F7F4CE4D875E87FF867C2DD98AC88ADE
:103CB0006F2D89890E94EA09811181CF80913C048E
:103CC000816080933C04C8010E948419DFCEFF20EC
:103CD00061F04D875E87FF867C2DD98AC88A6F2D5B
:103CE00089890E94EA0981116ACFC8010E9484195A
:103CF00070CF1F93CF93DF93CDB7DEB767970FB623
:103D0000F894DEBF0FBECDBF4B8B5C8B6D8B7E8B73
:103D10008F8B1A8A198A85E0FE017396DE011D9643
:103D200001900D928A95E1F786E0FE013D96DE0155
:103D3000179601900D928A95E1F7CE0107960E94A1
:103D4000E41C811137C086E0FE013796DE01119632
:103D500001900D928A95E1F79F8188852A853B85A0
:103D6000232B39F08F3F19F481E09F3F19F080E059
:103D700001C081E080FD1EC020913D0430E0C901FA
:103D800001968770992740916E044817190659F1DA
:103D900096E0929FD001939FB00D1124A25CBB4F7F
:103DA000FE01319601900D929A95E1F780933D04C2
:103DB0000E94E00916E080916E0490913D048917FD
:103DC000F9F0819FC0011124825C9B4F0E94E41C8A
:103DD0008823B1F080916E0490E001968770992756
:103DE00080936E04E8CF0E94C40F10923D0410929D
:103DF0006E0486E0E7E3F4E0DF011D928A95E9F7BF
:103E000067960FB6F894DEBF0FBECDBFDF91CF919E
:103E10001F9108958FEF84B980E485B9549A5C9A14
:103E20008FE19EE40197F1F700C0000008950F9321
:103E30001F93CF93DF938091E0039091E103209152
:103E4000F2033091F3033093E1032093E003909366
:103E5000F3038093F2035C9B0E940A1FD0E0C0E052
:103E600001E010E060E030E020E085B1422F807C8E
:103E70008C2B862B85B9EAE1EA95F1F700C0E09139
:103E8000E003F091E103EC0FFD1F808190E0022E32
:103E900002C0959587950A94E2F780FD2F9AF5E385
:103EA000FA95F1F7000076B52E988AE18A95F1F738
:103EB00000C0F80102C0EE0FFF1F4A95E2F7AF0104
:103EC0008091F2039091F303FC01EC0FFD1F4F9BD7
:103ED00075C0409550814523408346B5471B463009
:103EE00058F0E091E003F091E103EC0FFD1F4081F9
:103EF0008C0F9D1FFC014083FAE1FA95F1F700C099
:103F00002F982E9A8BE291E00197F1F700C0000004
:103F10002F5F3F4F685F2830310509F0A6CFA09191
:103F2000F203B091F303AC0FBD1FE091E003F091F9
:103F3000E103EC0FFD1F9C918081981751F00E94C6
:103F4000B5086093BE027093BF028093C002909345
:103F5000C1022196C830D10509F084CF5C9B28C0EE
:103F60008091B804853021F08091B804811120C07F
:103F70004091BE025091BF026091C0027091C10297
:103F80002FB7F8948091BA049091BB04A091BC041F
:103F9000B091BD042FBF841B950BA60BB70B8131CD
:103FA0009742A105B10520F00E94BE0C0E94CD08E9
:103FB00081E0DF91CF911F910F9108955081452BA2
:103FC0008BCFEF92FF920F931F93CF93DF93D82F56
:103FD0000E943E060FB607FE42C08091B8048430AE
:103FE00079F080910F0190E001962091110130E06D
:103FF00082239323209110012817190609F05FC02E
:104000008091DF0381110BC00E94B508643C7940A8
:104010008105910508F444C081E08093DF030E948C
:10402000C1088C01C091E900CF708091EC0080FD47
:1040300049C080E0C82B83E08093E90085E0E82E4A
:104040008091EB0085FD08C08091EB0080FF04C0EB
:104050008091EE0087FD56C0CF70C093E900E091DB
:104060000F018E2F90E001962091110130E0822304
:104070009323209110012817190609F494C0809108
:104080000D0190910E01E80FF92FF11DD083809161
:104090000F018F5F90911101892380930F0183C0DD
:1040A00080910F0190E001962091110130E0822370
:1040B0009323209110012817190609F4B0CFE0913D
:1040C0000F01DDCF80E8B6CFE0910D01F0910E0138
:1040D000E80FF11D90818F5F209111018223809361
:1040E00010019093F1008091E80085FD0BC0809154
:1040F000E80080FF07C08091E8008E778093E80099
:10410000E0920C018091100190910F01981741F1FC
:104110009091E80095FDD8CF80E029C01092F10081
:1041200032C080910F0190E001962091110130E0A2
:1041300082239323209110012817190609F08CCFB0
:10414000F0900C01FF2009F487CF0E94C10880176E
:10415000910709F475CFFA94F0920C018C0170CF9D
:104160008091E80085FFD8CFD093F10081E02091C5
:10417000F3009091F200322F292F232B79F09091A8
:10418000E80090FF0BC09091E80095FDC7CF90919B
:10419000E8009E779093E800E0920C01882309F2F2
:1041A000CF70C093E90080E0DF91CF911F910F9114
:1041B000FF90EF90089578941F920F920FB60F9290
:1041C00011248F939F93AF93BF938091BA049091E2
:1041D000BB04A091BC04B091BD040196A11DB11D0A
:1041E0008093BA049093BB04A093BC04B093BD0425
:1041F000BF91AF919F918F910F900FBE0F901F9025
:1042000018951F920F920FB60F9211248F939F93C0
:10421000AF93BF938091B904811113C08091BA0408
:104220009091BB04A091BC04B091BD044196A11D26
:10423000B11D8093BA049093BB04A093BC04B093C7
:10424000BD04BF91AF919F918F910F900FBE0F90C2
:104250001F9018951F920F920FB60F9211240F9373
:104260001F932F933F934F935F936F937F938F93FE
:104270009F93AF93BF93EF93FF93CF93DF93CDB70C
:10428000DEB7AA97DEBFCDBF1091E9001F70809105
:10429000EC0080FF3AC080E8182B1092E900809172
:1042A000F000877F8093F0007894EAE2F4E0809158
:1042B000F100819384E0E233F807C9F780912B0481
:1042C000833009F470C018F5813009F447C082309A
:1042D00009F4DAC08091E80083FF15C180912A04B7
:1042E00090912B049A3008F00EC1E92FF0E0E558C8
:1042F000FE4D0C94A32A55227B2283227B2283220B
:10430000F622182383221724242480E0C5CF8A3084
:1043100009F4A9C08B3009F47DC08930D9F68091A9
:104320002A048132B9F680912E0490912F04892BB2
:1043300089F68091E800877F8093E8008091E8000B
:1043400082FF2CC08091F100809306048091E800E8
:104350008B778093E8000E94380BBCCF80912A04B1
:10436000813A09F0B7CF8091E800877F8093E80019
:1043700080912E0490912F04892B61F060E090E0F1
:1043800080E070E00E94800A8091E8008B77809343
:10439000E800A0CF60E287E094E0F3CF8091B8041A
:1043A0008111CCCF97CF80912A04813A09F092CF26
:1043B00080912E0490912F04892BA1F48091E80024
:1043C000877F8093E8008091E80080FFFCCF809198
:1043D00028018093F1008091E8008E778093E800B7
:1043E0000E94380B80912E0490912F04019709F0C0
:1043F00071CF8091E800877F8093E8008091E8008A
:1044000080FFFCCF809126018093F1008091E8002D
:104410008E779FCF80912A04813209F05BCF809103
:104420002E0490912F04892B59F48091E800877F06
:104430008093E8000E94380B80912C04809328011F
:1044400080912E0490912F04019709F043CF809121
:10445000E800877F8093E8000E94380B80912C044D
:104460008093260137CF80912A04813209F032CF20
:104470008091E800877F8093E8000E94380B80914C
:104480002D048093C90426CF80912A04813A09F033
:1044900021CF8091E800877F8093E8008091E80039
:1044A00080FFFCCF8091C904AFCF803889F082387B
:1044B00051F580912E048F70873028F58093E900A4
:1044C0008091EB0085FB882780F91092E90006C0F7
:1044D0008091270490912804911182609091E800C6
:1044E000977F9093E8008093F1001092F100809103
:1044F000E8008E7749C0282F2D7F29F48823B1F159
:10450000823009F446C08091E80083FF0AC08091A0
:10451000E800877F8093E8008091EB0080628093C1
:10452000EB001092E9008091F00088608093F00029
:104530001F701093E900AA960FB6F894DEBF0FBE65
:10454000CDBFDF91CF91FF91EF91BF91AF919F913F
:104550008F917F916F915F914F913F912F911F911B
:104560000F910F900FBE0F901F90189580912C0403
:10457000813049F6933009F080E08093280410924E
:10458000E9008091E800877F8093E8000E94380B63
:10459000BACF80912C048111F2CF80912E048F70BC
:1045A0002FEF280F263008F0AECF8093E90020913E
:1045B000EB0020FFE4CF933031F48091EB00806278
:1045C0008093EB00DCCF9091EB0090619093EB0037
:1045D00021E030E001C0220F8A95EAF72093EA003B
:1045E0001092EA008091EB008860EACF81118BCFB6
:1045F00000912C040F778091E3008078802B8093CA
:10460000E3008091E800877F8093E8000E94380BE8
:104610008091E80080FFFCCF8091E3008068809368
:10462000E30083E0011101C082E08093B8046BCF06
:104630008058823008F067CF20912C0430912D04EF
:104640002C3DA3E03A07A1F583E08A838AE28983BF
:104650004FB7F894DE01139620E03EE051E2E32FDD
:10466000F0E050935700E49120FF03C0E295EF7013
:104670003F5FEF708E2F90E0EA30C0F0C7968D93C9
:104680009D932F5F243159F74FBF8091E800877FBA
:104690008093E8006AE270E0CE0101960E94800AF1
:1046A0008091E8008B778093E8002DCFC096E7CF0C
:1046B00080912E0490912F04432F552743305105AC
:1046C00009F44FC078F54130510509F445C084E53F
:1046D00090E0EEE8F4E04230510509F014CF20916B
:1046E000E800277F2093E8002091300430913104C6
:1046F0008217930708F49C0140E02115310509F069
:1047000063C0411161C08091E80082FDC9CF8091F2
:10471000B804882329F2853019F28091E80083FFDC
:10472000F2CFBECF4132510509F43FC042325105AC
:1047300009F0E9CE8330910508F0E5CEFC01EE0FDB
:10474000FF1FEB57FE4F0190F081E02D8E579E4FDB
:10475000DC018C9190E01DC082E190E0E2EEF4E09B
:10476000BECF332721303105C1F060F02230310552
:1047700009F0C9CEE4EFF4E0E4918E2F90E0E4EF8D
:10478000F4E007C0E8E1F5E0E4918E2F90E0E8E185
:10479000F5E0009709F4B7CEA2CFE8E0F5E0E491A8
:1047A0008E2F90E0E8E0F5E0F4CF8330910508F03B
:1047B000AACE880F991FFC01E557FE4F0190F081AA
:1047C000E02D89E090E08BCF8091B804882309F434
:1047D00067CF853009F464CF8091E80083FD60CF16
:1047E0008091E80082FD8FCF8091E80080FF85CF27
:1047F0008091F3009091F20089279827892721154D
:10480000310519F08830910550F041E0089709F022
:1048100040E08091E8008E778093E8006ECF44916D
:104820004093F1003196215031090196E8CF80384C
:1048300009F069CE8091E800877F8093E80080913D
:1048400029048093F10053CE81115DCE00912C0498
:10485000023008F058CE8091E800877F8093E8000E
:10486000009329040E94380B002399F084E0809380
:10487000B80442E261EC81E00E94570B42E061EC37
:1048800082E00E94570B46E261EC83E00E94570BE6
:104890003ACE8091E30087FDE9CF81E0E8CF1F9217
:1048A0000F920FB60F9211242F933F934F935F9364
:1048B0006F937F938F939F93AF93BF93EF93FF93E8
:1048C0008091E10082FF09C08091E20082FF05C073
:1048D0008091E1008B7F8093E1008091DA0080FF7E
:1048E0001FC08091D80080FF1BC08091DA008E7FAE
:1048F0008093DA008091D90080FFBAC080E189BD41
:1049000082E189BD09B400FEFDCF81E08093B80447
:1049100080910404811104C00E94420A0E94890B04
:104920008091E10080FF1FC08091E20080FF1BC0EA
:104930008091E2008E7F8093E2008091E2008061AE
:104940008093E2008091D80080628093D80019BCE7
:1049500085E08093B804809106048093050410924A
:1049600006040E94C40F8091E10084FF2DC0809155
:10497000E20084FF29C080E189BD82E189BD09B4DC
:1049800000FEFDCF8091D8008F7D8093D80080916C
:10499000E1008F7E8093E1008091E2008F7E809322
:1049A000E2008091E20081608093E200809129041E
:1049B000882309F463C084E08093B8040E94C40F84
:1049C00080910504809306048091E10083FF3FC03D
:1049D0008091E20083FF3BC08091E100877F80935C
:1049E000E10082E08093B804109229048091E100F4
:1049F0008E7F8093E1008091E2008E7F8093E200C1
:104A00008091E20080618093E20042E060E080E01B
:104A10000E94570B8091F00088608093F00081E045
:104A2000809328011092C9041092060480E2E7E006
:104A3000F4E0DF011D928A95E9F7EFE9F2E01192C7
:104A4000B2E0EE3BFB07D9F781E080932601FF91AE
:104A5000EF91BF91AF919F918F917F916F915F91F6
:104A60004F913F912F910F900FBE0F901F9018956F
:104A700019BC1092B8041092040452CF8091E30044
:104A800087FD02C081E098CF83E096CFCF93DF937C
:104A9000CDB7DEB72A970FB6F894DEBF0FBECDBFF5
:104AA00084B7877F84BF0FB6F894A8958091600083
:104AB000886180936000109260000FBE80E890E0F3
:104AC0000FB6F89480936100909361000FBE0E942E
:104AD000420A0E94890B8091E20084608093E20088
:104AE00081EE9FE190939D0180939C01509A589A8A
:104AF0005198599A78948FEF9091B80481509430DE
:104B000041F0EFE7FEE33197F1F700C000008111BB
:104B1000F3CF83E894E00E94810685B7806885BF63
:104B200085B7806885BF0E94F80B86988E9A819819
:104B30008998559A5D9888E08093CC001092CD00BA
:104B40008091C90080698093C9008091C900886004
:104B50008093C9008091CA008093CA008091CB00E5
:104B60008093CB00559A5D987894859A8D98FFEF45
:104B700021EE34E0F15020403040E1F700C0000069
:104B8000859A8D9A4FEF81EE94E04150804090409D
:104B9000E1F700C00000859A8D98EFEFF1EE24E078
:104BA000E150F0402040E1F700C00000859A8D9A66
:104BB0003FEF41EE84E0315040408040E1F700C0DB
:104BC000000085988D9880EC80937C0087E080932E
:104BD0007A0081E980937E0081E080937F008BE3FF
:104BE00080937D00849A8C988091270180930004A3
:104BF00087E794E00E94810682E084BD93E095BD42
:104C00009AEF97BD80936E008FEF84B980E485B9E9
:104C100057985F9A87B18F7387B988B1806C88B9CC
:104C20002E9A2F980E94BE0C1092EA031092EB036A
:104C30001092EC031092ED031092EE031092EF032A
:104C40001092F0031092F1031092E2031092E3032A
:104C50001092E4031092E5031092E6031092E7032A
:104C60001092E8031092E9038AEE93E09093F30325
:104C70008093F20382EE93E09093E1038093E0034C
:104C800087E694E00E948106F8E42F2EF4E03F2EA0
:104C9000ACE34A2E512C612C712C799B05C080917C
:104CA000B804853009F48DC10E94171FE5EFCE2EA0
:104CB000E3E0DE2EF12CE12C9E2CE091F203F0914A
:104CC000F303EE0DFF1DA080F601B080BA1409F4C5
:104CD00062C08091CB0481FF3CC08BE194E00E94D4
:104CE000810610E000E0E091F203F091F303E00FA1
:104CF000F11F2081229530E0C901880F991F880F8C
:104D0000991F8C7C35952795359527952373822B94
:104D100090E024E331E03F932F939C01220F331F57
:104D20002A7A959587958575822B1F928F931F936D
:104D30000F9380E194E09F938F930E941A070F5F77
:104D40001F4F0FB6F894DEBF0FBECDBF0830110560
:104D500051F600E011E0BA248B2D8123C1F00E83BF
:104D60009F8291E08A2D812309F490E098870E9428
:104D7000C1088160782F9A8789874E815F81688515
:104D80008A850E94791EF6018081812780830F5FCA
:104D9000110F083009F7FFEFEF1AFF0A2FEFC21AC1
:104DA000D20A38E0E316F10409F086CF8FEF898349
:104DB0008A831B820E94C1088160782F9D838C8327
:104DC00049815A816B818D810E94791E2091C20494
:104DD0003091C3044FB7F8948091BA049091BB040A
:104DE000A091BC04B091BD044FBFAC01421B530B5A
:104DF0008091BF0420912D0130E0811106C02091E7
:104E00002E019AE0299F900111244217530780F048
:104E10009091C5041091C604F090C7040091C80495
:104E20009111FBC01111D7C1F110D5C10111D3C12E
:104E30000E94360A9091F4038917D9F00E94360A2D
:104E40008093F4039091CB049570953061F41F9298
:104E50008F9388E294E09F938F930E941A070F909C
:104E60000F900F900F908091F403569A81FF43C1E9
:104E70005E9A82E0F82EEE24E39493E0D92E0E940D
:104E80009B0C8C01019609F038C1809102048111BC
:104E90001BC08091C0049091C10420910104211194
:104EA00072C1799970C18C51914071F00E94C40F08
:104EB0008091270180930004109227018CE191E0FA
:104EC0009093C1048093C0042091FE033091FF03AE
:104ED0004FB7F8948091BA049091BB04A091BC04A0
:104EE000B091BD044FBF821B930B893E43E09407F2
:104EF00008F460C028EE33E0B9010E94592A629F8D
:104F0000A001639F500D729F500D11248091FE03EC
:104F10009091FF03840F951F9093FF038093FE03EE
:104F20000E94CE12833009F03BC1859A8D980E9471
:104F3000B5086B017C0128EE33E040E050E00E94B0
:104F4000812A49015A01CA01B901A30192010E94B3
:104F5000812A672B682B692B69F50E949712209193
:104F6000CB0420FF27C09F938F931F921F92C501F0
:104F7000B40120E13EE040E050E00E94812AA3011C
:104F800092010E94812A3F932F93C701B60120E826
:104F90003EEE46E350E00E94812A1F922F9383E366
:104FA00094E09F938F930E941A070FB6F894DEBF88
:104FB0000FBECDBF7999F6C07E9BF4C06E9A7698ED
:104FC0006CCE83E694E00E9481060E94C40C0E948D
:104FD000CD080E94CD080E94CD080E94CD080E94F5
:104FE000CD080E94CD080E94CD0880912804882316
:104FF00009F453CE0E940A1F0E94171F0E94C40C7E
:10500000E091F203F091F303CF0108962191211171
:10501000CCC08E179F07D1F740CE8F3F19F08F5F1E
:105020008093BF04191624F40E94E0078093C504FE
:105030008091C50487FF05C00E94E0078195809399
:10504000C504111624F40E94E0078093C6048091E1
:10505000C60487FF05C00E94E00781958093C604BF
:105060006091C504662331F11091C604112311F13A
:10507000062E000C770B880B990B0E94602923E306
:1050800033E343E35FE30E94C4290E94282960932D
:10509000C504612F110F770B880B990B0E946029B3
:1050A00023E333E343E35FE30E94C4290E942829FA
:1050B0006093C6041F1424F40E94A7078093C704BA
:1050C0008091C70487FF05C00E94A7078195809340
:1050D000C704101624F40E94A7078093C804809187
:1050E000C80487FF05C00E94A70781958093C80464
:1050F0000E946F0E9DCE5E98BCCE809103048130DD
:1051000029F138F0823041F1833061F110920304CB
:10511000B6CE0E3F110519F4E0920304B0CE00386C
:10512000110568F41F930F93E0E6F4E0FF93EF930B
:105130000E941A070F900F900F900F90A0CE1F9310
:105140000F938AE594E09F938F93F2CF023011057D
:10515000E9F6F092030493CE01301105B9F6D0922E
:1051600003048DCE8091CB0480FF0AC01F930F9360
:105170003F922F920E941A070F900F900F900F905E
:105180000093FD03C3CF8251914009F49DCE0E944C
:10519000C40F809100048093270182E191E090CEBA
:1051A0008598C4CE6E9A769A78CD80E189BD82E1E9
:1051B00089BD09B400FEFDCF8091D8008F7D80931A
:1051C000D8008091E00082608093E0008091E00050
:1051D00081FDFCCF62CD8F3F09F021CF32CF1F92EE
:1051E0000F920FB60F9211242F933F934F935F931B
:1051F0008F939F93EF93FF938091C303E82FF0E089
:105200008F5F2091C203281739F09091CE00EE53A2
:10521000FD4F90838093C3033091C303432F50E02D
:10522000822F90E0841B950B321780F403970CF4C7
:105230005D9AFF91EF919F918F915F914F913F9177
:105240002F910F900FBE0F901F9018959395EECF52
:105250000E942F296894B1110C94BE2908950E94D0
:10526000A32988F09F5798F0B92F9927B751B0F02C
:10527000E1F0660F771F881F991F1AF0BA95C9F7DA
:1052800014C0B13091F00E94BD29B1E008950C9492
:10529000BD29672F782F8827B85F39F0B93FCCF345
:1052A000869577956795B395D9F73EF49095809557
:1052B000709561957F4F8F4F9F4F0895E89409C077
:1052C00097FB3EF490958095709561957F4F8F4F39
:1052D0009F4F9923A9F0F92F96E9BB279395F6954F
:1052E000879577956795B795F111F8CFFAF4BB0FCD
:1052F00011F460FF1BC06F5F7F4F8F4F9F4F16C031
:10530000882311F096E911C0772321F09EE8872FBA
:10531000762F05C0662371F096E8862F70E060E076
:105320002AF09A95660F771F881FDAF7880F9695EF
:10533000879597F9089557FD9058440F551F59F0D8
:105340005F3F71F04795880F97FB991F61F09F3F72
:1053500079F087950895121613061406551FF2CF9B
:105360004695F1DF08C0161617061806991FF1CFEB
:1053700086957105610508940895E894BB27662712
:105380007727CB0197F908950E94D7290C94482AD2
:105390000E943A2A38F00E94412A20F0952311F009
:1053A0000C94312A0C94372A11240C94BE290E94A3
:1053B0009B2970F3959FC1F3950F50E0551F629F95
:1053C000F001729FBB27F00DB11D639FAA27F00D5E
:1053D000B11DAA1F649F6627B00DA11D661F829F85
:1053E0002227B00DA11D621F739FB00DA11D621F6A
:1053F000839FA00D611D221F749F3327A00D611D87
:10540000231F849F600D211D822F762F6A2F112468
:105410009F5750409AF0F1F088234AF0EE0FFF1F9B
:10542000BB1F661F771F881F91505040A9F79E3FF2
:10543000510580F00C94312A0C94BE295F3FE4F3AF
:10544000983ED4F3869577956795B795F795E79548
:105450009F5FC1F7FE2B880F911D9695879597F951
:10546000089597F99F6780E870E060E008959FEFE6
:1054700080EC089500240A941616170618060906EB
:10548000089500240A9412161306140605060895BA
:10549000092E0394000C11F4882352F0BB0F40F442
:1054A000BF2B11F460FF04C06F5F7F4F8F4F9F4F82
:1054B0000895AA1BBB1B51E107C0AA1FBB1FA6175B
:1054C000B70710F0A61BB70B881F991F5A95A9F7AD
:1054D00080959095BC01CD01089597FB072E16F499
:1054E000009407D077FD09D00E94592A07FC05D007
:1054F0003EF4909581959F4F0895709561957F4FEB
:105500000895A1E21A2EAA1BBB1BFD010DC0AA1F04
:10551000BB1FEE1FFF1FA217B307E407F50720F01C
:10552000A21BB30BE40BF50B661F771F881F991F97
:105530001A9469F760957095809590959B01AC01E0
:10554000BD01CF010895EE0FFF1F0590F491E02DEE
:065550000994F894FFCF5E
:10555600F50BF00BF10BEF0BEE0B1C01059E01009A
:1055660000FFEA0B44121612D6119E11F20B750CAF
:105576005B0CED0B020C0101012808140A321E52C5
:105586004E2D3432004C554641004F464600434F9F
:105596004E4E004F4E00556E6174746163686564CB
:1055A60000506F77657265640044656661756C745A
:1055B6000041646472657373656400436F6E666967
:1055C60067757265640053757370656E6465640013
:1055D6003F00397F224D01CE00AC00A004B904D2B1
:0C55E60004010203040506070809000088
:106800000000000000000000040005000600070072
:10681000080009000A000B000C000D000E000F001C
:1068200010001100120013001400150016001700CC
:10683000180019001A001B001C001D001E001F007C
:10684000200021002200230024002500260027002C
:106850002800000035002B002C002D002E002F00FA
:1068600030002A00000033003400290036003700D1
:106870003800E00000000000000000000000000000
:106880000000000000000000000000000000000008
:1068900000000000000000000000000000000000F8
:1068A00000000000000000000000000000000000E8
:1068B00000000000000000000000000000000000D8
:1068C00000000000000000000000000000000000C8
:1068D00000000000000000000000000000000000B8
:1068E0000000000000000000310000000000000077
:1068F0000000E100E200E300F1A1E500E600E700AE
:106900000000000000000000EA4401000100E24431
:106910000100B84401005500460054004A004B00F5
:10692000560057004700480001000100E9440100FB
:106930000100010001000100010001003A003B00DC
:106940003C003D003E003F0040004100420043004B
:10695000580000004C00390001004400450052007E
:1069600001000100000050004F0081404D004E002A
:1069700051000100000000000000000000000000C5
:106980000000000000000000000000000000000007
:1069900000000000000000000000000000000000F7
:1069A00000000000000000000000000000000000E7
:1069B00000000000000000000000000000000000D7
:1069C00000000000000000000000000000000000C7
:1069D00000000000000000000000000000000000B7
:1069E000000000000000000049000000000000005E
:1069F0000000010001000100010001000100010090
:00000001FF
